:020000020000FC
:100000000C94CD000C943E000C943E000C943E00E9
:100010000C943E000C943E000C943E000C943E0068
:100020000C943E000C943E000C943E000C943E0058
:100030000C94A2000C943E000C943E000C943E00E4
:100040000C943E000C947A000C943E000C943E00FC
:100050000C9473000C943E000C946F000C943E00C2
:100060000C943E000C9466000C943E000C943F00EF
:100070000C943E000C943E000C943E0018953FB644
:100080000F931F93A0E0B4E02899549600917C0050
:10009000000F1127A00FB11F0D911D912801000F16
:1000A000111F040D151D4090780050907900040D2B
:1000B000151D0E5F1F4F16950795169507951E93F4
:1000C0000E93A99A1F910F913FBE18953FB6280134
:1000D00006E910E0600E711E82013FBE18951C9B60
:1000E0000E94FC0E18953090D200B3E0AF2D3D92E7
:1000F000FA2E18953FB60F9300917C000A950230B6
:1001000020F408D010D0189A0BE000937C000F91D7
:100110003FBE189588943099089400913904001FC7
:10012000009339040895839480FE0895F29A81FE25
:10013000089582FE0895F19A83FE089584FE08953D
:10014000F09A08953FB62B01609134047091350404
:10015000660D771D7695679560933404709335042A
:100160006624772466277091360467130FD065E004
:100170000E94F4032394271630F066E00E94F403F3
:100180007F7179BB2224B2013FBE18957A95709396
:100190003604671308950C94FC0E00E10EBF0FEFB8
:1001A0000DBFA895002704BF00916000086100936F
:1001B000600000270093600000270EBB09BB00E130
:1001C00005B901E004B900E808B902E007B902E0A6
:1001D0000BB907E80AB900E00EB900E00DB9F0E08C
:1001E000E6E0F093B300E093B200F695E795F09364
:1001F000B100E093B00008E00093B50000E8009380
:10020000BA0000E00093BB0000E20093B60001E0FA
:100210000093B700E8942224662477249924AA2422
:10022000C6D0BBD0BFD0B4D0EE24FF2400270093AB
:100230003C0400933D0400933E0400933F0400936C
:1002400040040027009336040093370400933804D9
:100250000FEF00933904002700933A0400933B0406
:100260000E9408100E9480100E94941069E00E9471
:10027000F4037F707ABB5F9BF49A112704E0D09B54
:100280000E942F1005E0D19B0E942F1006E0D29B08
:100290000E942F1007E0D39B0E942F1004E00093D0
:1002A0006D0000E100936A0009E00BBB0093680059
:1002B0000BE000937C000FEB00937A0002E20093C6
:1002C0007B000CEF00937E0007E000937F00002787
:1002D00004BD05BD00936E0006BD05E007BD03E04B
:1002E00005BD01E005BB00936E0000270093800070
:1002F0000093810000936F000093850000938400B9
:1003000011E607EA10938900009388000BE0009340
:10031000810002E006BB00936F006BD000270093C2
:10032000C8000FE90093CC000FE00093C80008E07C
:100330000093CD0000E00093CE0001E00093C900DF
:100340000093CA0000270093D200F1E2E8E35ED7F1
:1003500078D78CD7F3D778940091C90003FD00912A
:10036000D200FE100E941304F3990E94110900911B
:10037000DC0005FF0E9450020E94CF09F0990E9404
:10038000FA0CF1990E94B40EF2990E94DA0EE4CFB1
:100390000027E1E4F4E01BE128C00027ECE2F4E0F0
:1003A00014E023C00027E0E3F4E014E01EC00027BF
:1003B000E0E0F4E01CE219D000E012E000930C044D
:1003C00010930D0400931804109319040093200453
:1003D000109321040FEA10E0009316041093170401
:1003E00000932A0410932B04089501931A95E9F7BA
:1003F00008954427042F02950093ED0000270093F1
:10040000EE000093EF00242F2DD04395463090F35B
:1004100005E00093F40000E00093F50000E0009395
:10042000F6000EEF0093F7000FE70093DA0008E202
:100430000093DB0000E20093DE006BE00E94F40317
:1004400077FD7727770F7093E2000CE00093E300CD
:1004500006E31127711307E30093E40002E0009321
:10046000D80008956CE00E94F403072F6DE00E940D
:10047000F403172F3EE1000F111F221F331F000F3F
:10048000111F221F331F000F111F221F331F009344
:10049000F0001093F1002093F2003093F3000895E0
:1004A00000E50093ED000091DA0007FD07C000278A
:1004B0000093EE0000E90093EF0008950091EE0034
:1004C00011271093EE000E72003209F0089500918A
:1004D000F0001091F1002091F2003091F300369578
:1004E000279517950795369527951795079536956E
:1004F0002795179507956CE00E94F403071729F4D8
:100500006DE00E94F403171729F07FEF0717170714
:1005100009F008950091EF000F7081F0112402306E
:1005200011F018F008951090FA000090FA002F735F
:100530003327E6EAF2E0E20FF31F09942F73332723
:10054000E6E0F3E0E20FF31F8DDF099408950895CC
:1005500008950895089508950895089508950895B3
:100560000895089508950895089530C03DC5B6C50D
:10057000F0C577C51FC444C4E7C409C564C4EAC351
:10058000089581C3089508950895089521C02AC04B
:1005900030C039C0089508950895089508950895C4
:1005A0000895089508950895089508959BC40895A1
:1005B0000895089508950895089508950895089553
:1005C00008950895089508950895089509BA08951D
:1005D0000FE000220AB3007F00290ABBD19BF798E5
:1005E0001CD6ACC60FE000220AB300290ABB15D600
:1005F000A5C60FE0002200940AB300210ABBD19BDC
:10060000F7980BD69BC600FC48C2ABC13FC040C0A8
:1006100041C042C043C008950895089508950895C3
:10062000089508950895089508953AC03CC044C0BF
:100630004CC054C05CC064C06CC074C07CC084C07A
:1006400008958BC0089508950895089594C008955D
:10065000089599C0A1C0A2C059C2089508950895EF
:1006600008950895089508950895089599C0A6C01D
:100670000895089508950895089508950895089592
:10068000089508950895089508950895C89A0895BD
:10069000C99A0895CA9A0895CB9A0895CC9A089554
:1006A0000FE109BB089561E00E94F4037093FA0022
:1006B00001E50093EF00089563E00E94F403709356
:1006C000FA0001E50093EF00089562E00E94F40350
:1006D0007093FA0001E50093EF00089564E00E9432
:1006E000F4037093FA0001E50093EF00089565E0CC
:1006F0000E94F4037093FA0001E50093EF0008955F
:1007000066E00E94F4037093FA0001E50093EF00A5
:10071000089567E00E94F4037093FA0001E50093E6
:10072000EF00089568E00E94F4037093FA0001E579
:100730000093EF00089569E00E94F4037093FA00BB
:1007400001E50093EF0008956AE00E94F4037093BE
:10075000FA0001E50093EF0008956DE00E94F403B4
:100760007093FA006CE00E94F4037093FA0002E5C3
:100770000093EF0008950AB30F700093FA0001E5AB
:100780000093EF0008950027F49903950093FA0071
:1007900001E50093EF0008950C94F10E0C94FC0E0B
:1007A0006FE00E94F4037093FA006EE00E94F4037D
:1007B0007093FA0002E50093EF00089501E00093C2
:1007C000FA0001E10093FA000DE00093FA0005E061
:1007D0000093FA0007E00093FA0005EE0093FA0098
:1007E00006E50093EF000895F999FECF0F931F934C
:1007F0000FB71127F89412BD61BDF89A70B50FBFFD
:100800001F910F9108950F93072F0E94F40307176C
:1008100041F07727F89472BD61BD00BDFA9AF99A4C
:1008200078940F9108956F2D6E19653008F408952E
:10083000D3E0CE2D0881C3950062043641F0053621
:1008400039F0023731F0033729F0E394089503C0FB
:10085000A3C03CC16DC16C3008F408950881C395F4
:100860000062093649F50881C3950062033721F516
:100870000881C39500620136F9F40881C3950062CE
:100880000236D1F40881C39500620C36A9F40881C0
:10089000C3950062053681F40881C3950062003279
:1008A00059F40881C3950062013641F0023639F0EF
:1008B000073631F0003729F0E394089503C018C0DB
:1008C0003DC053C00881C39500620B3259F40881C2
:1008D000C3950062033731F40881C3950D3021F0D0
:1008E0000A3011F0E3940895EC2ED09896D426C5E2
:1008F0000881C3950062033639F40881C39500620C
:10090000013621F0023671F0E39408950881C39511
:100910000D3021F00A3011F0E3940895EC2ED298B6
:100920007CD40CC50881C3950D3021F00A3011F03C
:10093000E3940895EC2ED39870D400C50881C39534
:100940000062053659F40881C39500620E3631F411
:100950000881C3950D3021F00A3011F0E394089519
:10096000EC2EF4985F9A59D4E9C40881C3950062CB
:10097000013659F40881C3950062093731F40881C2
:10098000C3950D3021F00A3011F0E3940895EC2E58
:10099000D198F79842D4D2C46B3008F408950881F6
:1009A000C39500620E3621F50881C39500620136B9
:1009B000F9F40881C39500620236D1F40881C39529
:1009C00000620C36A9F40881C3950062053681F4F3
:1009D0000881C3950062003259F40881C395006212
:1009E000013641F0023639F0073631F0003729F090
:1009F000E394089503C018C03DC052C00881C39558
:100A000000620B3259F40881C3950062033731F458
:100A10000881C3950D3021F00A3011F0E394089558
:100A2000EC2ED09AFAD38AC40881C39500620336AB
:100A300039F40881C3950062013621F0023671F065
:100A4000E39408950881C3950D3021F00A3011F028
:100A5000E3940895EC2ED29AE0D370C40881C39534
:100A60000D3021F00A3011F0E3940895EC2ED39A62
:100A7000D4D364C40881C3950062053659F4088153
:100A8000C39500620E3631F40881C3950D3021F014
:100A90000A3011F0E3940895EC2EF49ABED34EC4BC
:100AA0000881C3950062013659F40881C39500623C
:100AB000093731F40881C3950D3021F00A3011F067
:100AC000E3940895EC2ED19AA8D338C4663008F484
:100AD00008950881C39500620536A9F40881C3957D
:100AE0000062033781F40881C3950062053659F42A
:100AF0000881C3950062043731F40881C3950D3035
:100B000021F00A3011F0E3940895EC2E0E94E00FDA
:100B10000E94F10F0E940210F894A89500916000C5
:100B200008610093600008E00093600078940895E5
:100B30000881C3950062053631F0083629F0043784
:100B400021F0E394089502C017C32CC36B3008F45E
:100B500008950881C3950062043791F40881C39514
:100B60000062003269F40881C3950062033651F0D7
:100B7000003799F00337D1F0043709F1063741F116
:100B8000E39408950881C3950062013671F102363D
:100B900069F1043761F1E39408950881C395006217
:100BA000003731F1033729F1E39408950881C395A3
:100BB00000620033F9F00E36F1F0E39408950881F5
:100BC000C39500620033C1F00537B9F0E39408958E
:100BD0000881C3950062013689F0023681F0003742
:100BE00079F0033771F0E39408950CC05FC08AC0B8
:100BF000B9C0E8C00AC135C189C1ABC1CDC109C204
:100C000045C27FC26D3008F408950881C395006223
:100C10000D33B1F50881C3950F70002E0AE0009ED8
:100C20000881C3950F70000E0AE0009E0881C395ED
:100C30000F701127000E111E8001000C111C000CFA
:100C4000111C000E111E000C111C0881C3950F70A1
:100C50001127000E111E8001000C111C000C111C2C
:100C6000000E111E000C111C0881C3950F70112776
:100C7000000E111E0881C3950D3021F00A3011F0CD
:100C8000E3940895EC2E6CE0702DBDDD6DE0712DC8
:100C9000BADD00270093D8000091D90002FDFCCFF7
:100CA00001E00093D800A5DBB8D2E0C20881C3956B
:100CB00000620237A1F40881C3950062003779F41D
:100CC0000881C39500620D3351F40881C3950F70FC
:100CD000002E0881C3950D3021F00A3011F0E39405
:100CE0000895EC2E6BE0702D8EDD00270093D80068
:100CF0000091D90002FDFCCF01E00093D80079DB20
:100D00008CD2B4C26C3008F408950881C395006297
:100D10000D33E9F40881C3950F70002E0AE0009EA0
:100D20000881C3950F70000E0AE0009E0881C395EC
:100D300000620E3261F40881C3950F701127000E16
:100D4000111E0881C3950D3021F00A3011F0E39493
:100D50000895EC2E702D112009F07FEF6AE053DD2D
:100D60005CD284C26C3008F408950881C395006297
:100D70000D33E9F40881C3950F70002E0AE0009E40
:100D80000881C3950F70000E0AE0009E0881C3958C
:100D900000620E3261F40881C3950F701127000EB6
:100DA000111E0881C3950D3021F00A3011F0E39433
:100DB0000895EC2E702D112009F0772765E023DDD2
:100DC0002CD254C20881C39500620D33B1F408815E
:100DD000C3950F70002E0AE0009E0881C3950F7026
:100DE000000E0AE0009E0881C3950F70000E088176
:100DF000C3950D3021F00A3011F0E3940895EC2EE4
:100E000066E0702D00DD09D231C20881C395006211
:100E10000D33B1F40881C3950F70002E0AE0009ED7
:100E20000881C3950F70000E0AE0009E0881C395EB
:100E30000F70000E0881C3950D3021F00A3011F0BB
:100E4000E3940895EC2E69E0702DDDDC76FFF698D2
:100E5000F79B04C075FD02C0D19AF798DED106D287
:100E60006DC26D3008F408950881C39500620D339A
:100E7000B1F50881C3950F70002E0AE0009E08812D
:100E8000C3950F70000E0AE0009E0881C3950F7095
:100E90001127000E111E8001000C111C000C111CEA
:100EA000000E111E000C111C0881C3950F70112734
:100EB000000E111E8001000C111C000C111C000EF4
:100EC000111E000C111C0881C3950F701127000E14
:100ED000111E0881C3950D3021F00A3011F0E39402
:100EE0000895EC2E6EE080DC872F6FE07DDC972F7D
:100EF000019621F0C001019609F008956EE0702D71
:100F000082DC6FE0712D7FDC88D19BC10881C395A5
:100F100000620D33B1F40881C3950F70002E0AE012
:100F2000009E0881C3950F70000E0AE0009E0881A4
:100F3000C3950F70000E0881C3950D3021F00A3063
:100F400011F0E3940895EC2E67E0702D5CDC65D120
:100F50008DC10881C39500620D33B1F40881C3953A
:100F60000F70002E0AE0009E0881C3950F70000EDE
:100F70000AE0009E0881C3950F70000E0881C3959A
:100F80000D3021F00A3011F0E3940895EC2E68E062
:100F9000702D39DC42D16AC16C3008F408950881A3
:100FA000C39500620D33E9F40881C3950F70002EDC
:100FB0000AE0009E0881C3950F70000E0AE0009EB3
:100FC0000881C39500620E3261F40881C3950F70E9
:100FD0001127000E111E0881C3950D3021F00A3033
:100FE00011F0E3940895EC2E06E710E000161106C8
:100FF00010F4702F08C000EF10E00015110510F478
:10100000702F01C0702D61E0FEDB0E94801005D1C1
:101010002DC16C3008F408950881C39500620D332A
:10102000E9F40881C3950F70002E0AE0009E088144
:10103000C3950F70000E0AE0009E0881C395006200
:101040000E3261F40881C3950F701127000E111E36
:101050000881C3950D3021F00A3011F0E394089512
:10106000EC2E05E810E00016110610F4702F08C0F1
:101070000CEF10E00015110510F4702F01C0702D59
:1010800064E0C1DB0E949410C8D0F0C06C3008F45A
:1010900008950881C39500620D33E9F40881C39572
:1010A0000F70002E0AE0009E0881C3950F70000E9D
:1010B0000AE0009E0881C39500620E3261F4088147
:1010C000C3950F701127000E111E0881C3950D30B6
:1010D00021F00A3011F0E3940895EC2E06E710E0B9
:1010E0000016110610F4702F08C000EF10E0001574
:1010F000110510F4702F01C0702D63E084DB8DD0DA
:10110000B5C06C3008F408950881C39500620D33B2
:10111000E9F40881C3950F70002E0AE0009E088153
:10112000C3950F70000E0AE0009E0881C39500620F
:101130000E3261F40881C3950F701127000E111E45
:101140000881C3950D3021F00A3011F0E394089521
:10115000EC2E03E210E00016110610F4702F08C008
:1011600008E710E00015110510F4702F01C0702D74
:1011700062E049DB52D07AC00881C39500620F3625
:1011800059F40881C3950062073731F40881C3958B
:101190000D3021F00A3011F0E3940895EC2E3DD08B
:1011A00065D0CCC00881C3950062013621F00F36AE
:1011B000C9F0E3940895663008F408950881C39552
:1011C0000062023759F40881C3950062043731F494
:1011D0000881C3950D3021F00A3011F0E394089591
:1011E000EC2EFFC50881C3950062003731F40881F9
:1011F000C3950D3021F00A3011F0E3940895EC2EE0
:10120000FBC5059109930023E1F70895D1E0C0E003
:10121000F8DFD1E0C0E06E01F39AF39B089501D0AE
:10122000FCCFE6010991002311F4F3980895109181
:10123000C90014FD089511FF08950093D2006E01B6
:101240000895F2E2EEE8D1E0C0E0DBDFF1E06EE02D
:101250000E94F403272F6FE00E94F403372FEFE082
:10126000AFD3D1E0C0E06E01F39AD7CFF2E2E6EA65
:10127000D1E0C0E0C6DFF1E061E00E94F403272F77
:101280003327EBE1A3D3B2D363E00E94F403272F0B
:101290003327E5E29BD3AAD362E00E94F403272F11
:1012A0003327EFE293D3A2D364E00E94F403272F05
:1012B0003327E9E38BD39AD365E00E94F403272F09
:1012C0003327E3E483D392D366E00E94F403272F0D
:1012D0003327EDE47BD367E00E94F403272F332705
:1012E000E5E574D368E00E94F403272F3327EDE58A
:1012F0006DD369E00E94F403272F3327E6E666D317
:101300006AE00E94F403272F3327EEE65FD36ED303
:101310006BE00E94F40320E3270FEAE721936CE0DF
:101320000E94F403272F6DE00E94F403372FE0E8BA
:1013300047D3D1E0C0E06E01F39A6FCFF3E2EEE263
:10134000D1E0C0E05EDFF1E0E6E1D09917D0E4E261
:10135000D09914D0E2E3D19911D0E2E3F7990ED0FD
:10136000E0E4D2990BD0EEE4D39908D0ECE5F499FF
:1013700005D0D1E0C0E06E01F39A4FCF25E4219370
:101380002EE6219321E6219322E621932CE6219358
:1013900025E6219324E6219320E22193089509B3C1
:1013A0000F7109F40895D1E0C0E0C8990FD0C99930
:1013B00024D0CA9938D0CB9948D0CC995BD0D1E011
:1013C000C0E06E01F39A002709BB08956E01F1E2B7
:1013D000E6E817DF92D0A4D1A3D0B4D1D2D0E5D122
:1013E00037D1CA950091DC0000FD089500E000931C
:1013F000ED0017E0E1E4F4E04FC06E01F1E2E0ED52
:1014000000DF57D05DD167D079D19DD0B0D1CA95DA
:101410000091DC0001FD089500E10093ED0016E06D
:10142000E8E4F4E039C06E01F2E2E4E1EADE1AD267
:1014300055D2CA950091DC0002FD089500E20093A8
:10144000ED0014E0EEE4F4E027C06E01F2E2E4E324
:10145000D8DE10D1A9D0BCD1D1D0E4D1CA950091A9
:10146000DC0003FD089500E30093ED0015E0E2E5E4
:10147000F4E012C06E01F2E2E8E6C3DE6BD278D28D
:10148000CA950091DC0004FD089500E40093ED008E
:1014900015E0E7E5F4E000C000270093EE0021919D
:1014A0002093FA0003950113FACF10651093EF0013
:1014B0000895F8940091040410910504789459E378
:1014C000159F9001059F210D20934804F601ED5FC3
:1014D000FF4F7CD28BC2F894009106041091070450
:1014E000789459E3159F9001059F210D20934A049C
:1014F000F601E75EFF4F6AD279C2F89420910804A2
:101500003091090478942F5F3F4F36952795369593
:10151000279520934104F601ED5FFF4F57D266C235
:10152000F89420910A0430910B0478942F5F3F4F78
:10153000369527953695279520934304F601E85E66
:10154000FF4F44D253C2F89400910C0410910D0443
:10155000789420E032E029D2F601E25DFF4F41931A
:1015600021E030E0200F311F3695279536952795DD
:10157000022F0F774B3209F0019500934C0426D2CD
:1015800035C2F89420910E0430910F0478942F5FA7
:101590003F4F369527953695279520934504F601BC
:1015A000E35DFF4F13D222C2F89400911004109112
:1015B00011047894133018F00BE410E00BC027ED01
:1015C00030E00217130728F025E332E00217130773
:1015D00008F0890121E431E0E8D1F601E35FFF4F33
:1015E000419356E8159F9001059F210D022F0F771B
:1015F0004B3209F0019500935304E8C1F89400912F
:101600001204109113047894133018F00BE410E0D6
:101610000BC027ED30E00217130728F025E332E076
:101620000217130708F0890121E431E0BED1F60169
:10163000EE5DFF4F419356E8159F9001059F210DE8
:10164000022F0F774B3209F0019500935504BEC16C
:10165000F89420911404309115047894890116951A
:1016600007951695079500934704F601EE5BFF4F2B
:10167000ADD1BCC1F89400911604109117042091CB
:101680002A0430912B047894020F131F67E00E9404
:10169000F40366272FED30E0270F361F86D1F601C1
:1016A000EE5FFF4F41935DEC159F9001059F210D6B
:1016B000022F0F774B3209F001950093520486C137
:1016C000F8940091180410911904789420E032E005
:1016D0006CD1F601E25FFF4F419321E030E0200F33
:1016E000311F3695279536952795022F0F774B3268
:1016F00009F001950093490469D178C1F8940091EB
:101700001A0410911B04789456E4159F9001059FCC
:10171000210D20934B04F601ED5DFF4F57D166C1BB
:10172000F89420911C0430911D04789436952795E7
:1017300089011695079500934204F601E25FFF4F79
:1017400045D154C1F89420911E0430911F0478941F
:101750002D5F3F4F369527953695279536952795DA
:1017600020934404F601EE5DFF4F30D13FC1F89461
:101770000091200410912104789420E032E015D1EA
:10178000F601E65CFF4F419321E030E0200F311F6E
:101790003695279536952795022F0F774B3209F00E
:1017A000019500934D0412D121C1F8942091220497
:1017B0003091230478942F5F3F4F369527953695C7
:1017C000279520934604F601E85CFF4FFFD00EC139
:1017D000F89400912404109125047894133018F0A3
:1017E0000BE410E00BC027ED30E00217130728F0E0
:1017F00025E332E00217130708F0890121E431E004
:10180000D4D0F601E85EFF4F419356E8159F900152
:10181000059F210D022F0F774B3209F001950093A0
:101820005404D4C0F89400912604109127047894AD
:101830002DEB31E00217130708F089012DE730E0A6
:10184000B4D0F601E45DFF4F419356E6159F900139
:10185000059F210D022F0F774B3209F00195009360
:101860005604B4C000912C0410912D0420912E0434
:1018700030912F044BE233234AF4015010402040B2
:10188000304000951095209530954DE2F601EC5FC3
:10189000FF4F419355E9772788279927059F612DA9
:1018A000159F600D711D259F700D811D359F800D49
:1018B000911D9695879577956795969587957795D8
:1018C0006795272F382F4B3221F0709580957F5FD9
:1018D0008F4F80934E0470934F0472C00091300478
:1018E0001091310420913204309133044BE23323C0
:1018F0004AF401501040204030400095109520954A
:1019000030954DE2F601ED5EFF4F419355E97727A3
:1019100088279927059F612D159F600D711D259FB3
:10192000700D811D359F800D911D9695879577953A
:1019300067959695879577956795272F382F4B3222
:1019400021F0709580957F5F8F4F80935004709346
:10195000510436C0F89420913404309135047894C1
:101960003093570420935804F601ED5FFF4F28C0D1
:101970002EB320935904F601E05FFF4F332726D0A2
:1019800026B120951C9B2F7720935A04F601E85E20
:10199000FF4F33271BD02AB3F799226020935B04B3
:1019A000F601E05EFF4F332711C0021B130B14F04A
:1019B0004BE2089501501040009510954DE20895B6
:1019C00017E200E109D013E008EE06D0112704E683
:1019D00003D00AE001D001E040E34395201B310B26
:1019E000E0F7200F311F4A954193089540834EE25E
:1019F00042930895F09805D014D175D17ED196D137
:101A00000895F894009116041091170420912A0467
:101A100030912B047894020F131F67E00E94F403A7
:101A200066272FED30E0270F361F021B130B9CF0AB
:101A30005DEC159F9001059F210D68E00E94F40365
:101A4000672F669566956695761B271720F0760FAB
:101A5000271718F40895F5980895F5990895F59ABB
:101A60005F9A0895F8940091040410910504209160
:101A70000804309109047894029FA001139FB001DB
:101A8000039F500D611D129F500D611D79E3479F0B
:101A90008001679F9001579F7727100D211D371FE9
:101AA0003695279517950795369527951795079598
:101AB000810F921FF89400911A0410911B04209139
:101AC0001E0430911F047894029FA001139FB0015F
:101AD000039F500D611D129F500D611D73E2479FC2
:101AE0008001679F9001579F7727100D211D371F99
:101AF0003695279517950795369527951795079548
:101B0000810F921FF8940091060410910704209110
:101B10000A0430910B047894029FA001139FB00136
:101B2000039F500D611D129F500D611D79E3479F6A
:101B30008001679F9001579F7727100D211D371F48
:101B400036952795179507953695279517950795F7
:101B5000810F921FF89400910C0410910D042091B4
:101B60000E0430910F0478941250B4F0029FA0013B
:101B7000139FB001039F500D611D129F500D611DF9
:101B800070E1479F8001679F9001579F7727100D55
:101B9000211D371F810F921FF8940091200410918E
:101BA0002104209122043091230478941250B4F03F
:101BB000029FA001139FB001039F500D611D129F52
:101BC000500D611D70E1479F8001679F9001579FF5
:101BD0007727100D211D371F810F921FF894009158
:101BE00018041091190420911C0430911D0478945C
:101BF0001250B4F0029FA001139FB001039F500D3B
:101C0000611D129F500D611D70E2479F8001679F0B
:101C10009001579F7727100D211D371F810F921FAD
:101C200008955F993BC080E197E21CDFF8944091F2
:101C30001404509115047894662771E6479F80013B
:101C4000679F9001579F7727100D211D371F801721
:101C50009107620760F480913A0490913B040197E8
:101C600097FD089580933A0490933B0408958091E2
:101C70003A0490913B0409960EE011E08017910719
:101C800028F480933A0490933B04089569E00E94FD
:101C9000F40376FF0895F69A5F9A089580913A04C6
:101CA00090913B0401972AF080933A0490933B046F
:101CB000089580E197E2D6DEF894409114045091A3
:101CC00015047894662771E6479F8001679F90010D
:101CD000579F7727100D211D371F80179107620727
:101CE00000F0F6980895F49B0895F5990895F699F3
:101CF0000895589908955F980895009137040395C1
:101D0000073B28F4009337040E3A38F4089500276F
:101D10000093370400933804089569E00E94F403A7
:101D200074FF08950CE0009338040895F89420910E
:101D30001C0430911D04789436952795332341F087
:101D40002A3008F40895F79B0895D19AF7980895DA
:101D5000F7990895D19B089569E00E94F40375FFF7
:101D60000895D198F79A0895F19807D001D0089571
:101D7000CCE0D4E0ECE2F4E005C0C0E2D4E0E0E383
:101D8000F4E000C0008111812281338140E052E003
:101D90006627041B150B260B360BF89448815981D6
:101DA0007894040F151F261F361F0083118322838A
:101DB00033830895F2980BD021D0092D3AD0091120
:101DC000A7D10A2D44D00A11AAD14FD0089500916D
:101DD0003904002319F0009561F008950EF4089578
:101DE00068945F9A589A6AE00E94F40370933604EC
:101DF00008950EF00895E89458980895F894209165
:101E00001C0430911D0478943695279500E713E063
:101E1000021B130B169507951695079516950795B2
:101E200016950795201B310B30FD2FEF37FD22272C
:101E3000089562E00E94F403972E291508F0089592
:101E4000922E13E2911608F00895912E089563E002
:101E50000E94F403A72E2A1508F00895A22E16E773
:101E6000A11608F00895A12E089523D00AB3109169
:101E700038041C7010950123102F12951095012322
:101E8000542F50231FE05123402B10EF4123452BAB
:101E900040FD7AD041FD89D042FD98D043FDA7D0C6
:101EA00044FD7DD045FD8CD046FD9BD047FDAAD09A
:101EB0000895F89420911C0430911D04789436956F
:101EC000279564E00E94F403072F11270E5E1F4F31
:101ED0002017310718F039D04FE0089500270093FC
:101EE0003C04072F11272017310718F034D043E0A6
:101EF0000895002700933D0411EE719F012D1127D5
:101F00002017310718F02DD043EC089500270093D7
:101F10003E0413EC719F012D11272017310718F093
:101F200026D040EC0895002700933F0415EA719FE6
:101F3000012D11272017310718F01FD040EE08950A
:101F400000270093400440EF089500913C0403955E
:101F500007FF00933C0400913D04039507FF0093A5
:101F60003D0400913E04039507FF00933E04009159
:101F70003F04039507FF00933F040091400403953D
:101F800007FF00934004089500913E04083108F4CF
:101F900008951FEF04E00E942F10D49A089511278E
:101FA00004E00E942F10D498089500913E0400335D
:101FB00008F408951FEF05E00E942F10D59A0895A8
:101FC000112705E00E942F10D598089500913C0438
:101FD000083408F408951FEF06E00E942F10D69AE7
:101FE0000895112706E00E942F10D69808950091B9
:101FF0003C04003608F408951FEF07E00E942F10FC
:10200000D79A0895112707E00E942F10D7980895B6
:102010005998419A5A9A4198419A5A984198419AA6
:102020005A984198419A5A9A4198419A4198419AAE
:102030004198419A4198419A4198419A4198419AD0
:102040004198419A4198419A4198419A4198419AC0
:102050004198419A4198419A4198599A08955998BE
:10206000419A5A984198419A02FF5A9802FD5A9A09
:102070004198419A01FF5A9801FD5A9A4198419A14
:1020800000FF5A9800FD5A9A4198419A17FF5A98B2
:1020900017FD5A9A4198419A16FF5A9816FD5A9A76
:1020A0004198419A15FF5A9815FD5A9A4198419ABC
:1020B00014FF5A9814FD5A9A4198419A13FF5A985E
:1020C00013FD5A9A4198419A12FF5A9812FD5A9A52
:1020D0004198419A11FF5A9811FD5A9A4198419A94
:1020E00010FF5A9810FD5A9A4198419A4198419A86
:1020F0004198419A4198419A4198599A5A9808951D
:1021000061E00E94F40315E7171B110F00E0A7CF51
:1021100018E71919712F110F170F01E0A0CF15E75C
:102120001A19110F02E09BCF64E00E94F40314E837
:10213000171B110F03E093CF0D0A4D696C6C737779
:102140006F6F6420456E67696E656572696E6720A2
:102150003235305720506F776572204D616E616760
:10216000656D656E7420556E69740D0A4669726DF1
:10217000776172652076657273696F6E3A20312ED1
:1021800031370D0A000056613D2A2A2E2A5620209A
:102190005632383D2A2A2E2A56202056703D2A2AA9
:1021A0002E2A56202056733D2A2A2E2A56202056A3
:1021B00062613D2A2A2E2A5620205662623D2A2A32
:1021C0002E2A56202056673D2A2A2E2A560D0A000E
:1021D00049613D2A2A2E2A4120204932383D2B2AA6
:1021E0002A2E2A41202049703D2A2A2E2A412020C9
:1021F00049733D2A2A2E2A4120204962613D2B2A1B
:102200002A2E2A4120204962623D2B2A2A2E2A4169
:102210000D0A00004562613D2B2A2A2A2A2A6D41B7
:102220004820204562623D2B2A2A2A2A2A6D4148ED
:102230000D0A0000543D2B2A2A2A432020546261B3
:102240003D2B2A2A2A4320205462623D2B2A2A2A27
:1022500043202054673D2B2A2A2A43202054653DE1
:102260002B2A2A2A430D0A0053673D2A2A2A2A2AA2
:1022700052504D202052303D2A2A2A202052313DF2
:102280002A2A2A202052323D2A2A2A0D0A00536582
:102290007269616C206E756D6265723A202A2A2A15
:1022A0002A2A0D0A0000436F6E66696775726174B1
:1022B000696F6E2073657474696E67733A20566136
:1022C0003D2A2A2E2A56202056703D2A2A2E2A568A
:1022D000202056733D2A2A2E2A56202056623D2A57
:1022E0002A2E2A56202050703D2A2A2E2A5320209A
:1022F00050733D2A2A2A202054303D2A2A2A2020A1
:1023000054753D2A2A2A43202053303D2A2A2A2068
:102310002043543D2A2A2E2A532020436272703DC6
:102320002A202043613D2A2A2A2A2A0D0A00456EC6
:1023300061626C65642066656174757265733A20CC
:102340004176693A44697361626C65642020536523
:10235000723A44697361626C656420205061793A15
:1023600044697361626C656420204243413A446968
:102370007361626C656420204243423A4469736130
:10238000626C6564202047656E3A44697361626CD3
:0623900065640D0A000067
:00000001FF
